:1000000022C088C179C189C188C187C172C1F0C0CD
:1000100084C183C182C181C180C1763330F101AB1B
:10002000FA00FA22B9AB63CBDBA2FBEB64003C0025
:1000300028001400140100D9133BD85B11005BF3B6
:100040005900010101016624DD27FF2702E00EBFF0
:100050000FE50DBF0FE168BA07BB01E201BB00E08D
:1000600002BB00EC0BBF0BE005BF03E003BF02E8DF
:1000700009BF0FEF02BF01E20FBD01E00EBD68BC7A
:100080007724442708E101BD0AE101BD78947DD1C0
:10009000F8D2B3FCFBD200918900001F00938B00C3
:1000A00001E00093660000270093670001E00093E1
:1000B0006800009369009AD000E008BD08E2D62CE1
:1000C000E02E63D1609270006092800050D294D193
:1000D000BB20F1F708E008BB1127139505E0B0FE3F
:1000E00002C0C6E609C01127B1FE02C0C7E604C0BF
:1000F000B2FE09C0C8E602E0F880F394F01608F0FA
:10010000F12EF882DFCFC9E6B3FE04C00EE111E0A4
:10011000BCD1DDCFB4FE04C001E01FEFB6D1D7CF14
:10012000B5FC03C0D9CF44274EC096D205E0E016F7
:100130000CF4E02EC9E60991099300E0099304E06C
:10014000088315D2AA24FF2700916700002309F035
:1001500003950395302F00916600102F002309F4BA
:100160003FEF0A95363019F40370086008BB07E0CA
:10017000100FC8D2902E7894BB20F1F7E2E4D0D1D2
:10018000432FCBE608810A950F3F39F4CA950881C1
:100190000A9509930F3FB9F00BE30883CA9548D13C
:1001A000A8EEB3E0B6FC0FC0B7FFFCCF009168002B
:1001B000002339F700916B00027019F44F3F01F3EF
:1001C000E0CF4FEFDECF4FEF08E2D62CE02EE6E394
:1001D000B6FEB6D1A4E6B0E0B7FFFECF60927000E5
:1001E0004427A4E6B0E0B7FFFECF6CCF2AD2089533
:1001F0004FB60F930FEF02BF442311F18A9489F495
:1002000009E1802E53954530F9F14630F1F04F3F2A
:10021000A9F15B3431F443955FE5959860927000E5
:10022000A8957CD05A9449F40DE7502E772009F018
:100230007A9459D0B7FF119778D00F914FBE189587
:10024000909A9598C498A895ECCF0E2D0230A4F4FE
:10025000C49AEE2089F400916600002341F00091D9
:100260007000869B0064879B006200937000513091
:1002700019F4909860927000A895D3CF909A9598B1
:10028000A89560927000CDCFC398959B05C0C3948C
:10029000C91411F49598A895593119F4CC24959A5C
:1002A000C0CF563419F49598A895BBCF5B3411F4A0
:1002B0009098B7CF5C3411F4909AB3CF5B3490F040
:1002C0005F3564F400916600002341F000917000F6
:1002D000869B0064879B0062009370005A3509F08A
:1002E000A0CF432F9ECFEE2019F0DA9409F4EA94C0
:1002F00008954FB60F93A1CF4FB60F935A3548F0DC
:10030000562D00917000009380006092700001E013
:10031000802E93CF4FB60F9390CFFFCF772011F061
:10032000C29A0895C298089508950FEF6ABA0BBB58
:100330006395770F663010F0662771E000E404BB28
:10034000CF93C0E6C60F0881C9B36BBA74BB0ABBB2
:10035000C09500917400C01729F0C093740000E5A7
:1003600000937300009173000A9519F40395B090FF
:1003700074000093730000916500C09180000F71BC
:100380000C2B00936500CF91089506E001C004E0B6
:10039000C0E669920A95E9F708950395FF24089449
:1003A000FF1C0A95E9F70F2D0895102F0F70065FB7
:1003B0001051E8F70A500895FF240A5010F0F39402
:1003C000FCCF065F0895F8DFFF0CFF0CFF0CFF0C5D
:1003D0000F290895F1DF02D0102F0F2DEF93E2E2E5
:1003E000E00FC895002DEF91089500918C00D5DFA6
:1003F00000936400088112C000916700CEDF009373
:10040000650000916600C9DF102F009168000B5F46
:10041000C4DF012B009364000091690060926300C7
:1004200060926200D7DF009361001093600008952E
:100430000991D0DF00936300109362000991CADF35
:10044000F9900F291F29009361001093600008950F
:10045000F22C0881031521F0010D0883FA94C9F7E5
:10046000F214089500D0A82FBB27BB208894C9F3AD
:10047000B7FFFBCF08940895EBDF08F478D0CEDF08
:10048000F1DF78F79A95C1F70895112E302E8FEF8E
:1004900091E0292EF1DF60F48EE695E0EDDF40F487
:1004A0009CE080E5E9DF20F49AE08DE2E5DFE0F30F
:1004B0000895F22C0881010D07FF02C0032D0A9553
:1004C000031509F400270883FA94A1F7089500D0D2
:1004D000A82FBB27BB208894C9F3B7FFFBCF089494
:1004E0000895E7DF44D0CF93CDE6A2DFCF91EFDFD1
:1004F00068F79A95B1F70895112E302E8FEF91E09D
:10050000292EEFDF60F48EE695E0EBDF40F49CE00F
:1005100080E5E7DF20F49AE08DE2E3DFE0F3089581
:10052000C89500926300E395C89500926200E39538
:10053000C89500926100E395C89500926000089507
:10054000EFDF10E11F930FEF702EA8EEB3E0BB209A
:1005500011F4B7FFFCCF1F91BB2041F41A9591F71E
:10056000AFEFBFE7BB2011F4B7FFFCCF08950F93A7
:1005700009E1702E0F91089520E12A95F1F7089571
:1005800028E02A95F1F708958E9A8F98F5DF8E98D6
:10059000F7DF082F8F9AF4DF0894001F01C0000FC7
:1005A00059F08E9A18F400008F9802C08F9A00C0FC
:1005B000E3DF8E98E1DFF3CF8E9A8F98DDDF8E98A0
:1005C000869BFECF889487990894D6DF089580FF94
:1005D000E3CF991F01E08E9ACFDF8E98CDDF88940C
:1005E00087990894001FB8F78E9A979510F48F9802
:1005F00001C08F9AC1DF8E98869BFECFBDDF089524
:100600008E9A8F9AB9DF8E98BBDF8F98B5DF0895E9
:10061000969897988E988F98089580EDBADF0F2D51
:10062000D6DF012FD4DFECDF08952F9380EDB1DF0B
:100630000F2DCDDF81EDA8DF0894C9DFE1DF2F9119
:10064000089504E0F02EDD27C6E613E05BD00993A1
:100650001395FA94D9F7089504E0F02EDD27C6E645
:1006600013E0099147D01395FA94D9F708952227FA
:1006700018E0069508F42F0D279507951A95D1F7E0
:100680000895A4E6B0E0B7FFFECF0895EDE158DF8E
:10069000A8EEB3E0B6FC02C0B7FFFCCF089539D096
:1006A000EAE34EDFB3FCFECF01E000938C005FDF96
:1006B00000918C00C5E7C00F98DEBB20F1F7B0FEBB
:1006C00009C000918C000395053008F001E000930B
:1006D0008C00EDCFB3FE04C00CE311E0D6DEE8CF12
:1006E000B4FE04C001E01FEFD0DEE2CFB5FC01C0D4
:1006F000E6CF15C0E199FECF6FBA1EBB0DBBE29AE3
:10070000E19A0895E199FECF6FBA1EBBE09A0DB34E
:10071000089504E0F02EDD27C6E718E097CF04E047
:10072000F02EDD27C6E718E09CCFFFFFFFFFFFFF9D
:102000005050800400010100141E2532FFFFFFFF25
:10201000FFFFFFFFFFFFFFFFFFFFFFFFFFFFFFFFD0
:10202000FFFFFFFFFFFFFFFFFFFFFFFFFFFFFFFFC0
:10203000FFFFFFFFFFFFFFFFFFFFFFFFFFFFFFFFB0
:10204000FFFFFFFFFFFFFFFFFFFFFFFFFFFFFFFFA0
:10205000FFFFFFFFFFFFFFFFFFFFFFFFFFFFFFFF90
:10206000FFFFFFFFFFFFFFFFFFFFFFFFFFFFFFFF80
:10207000FFFFFFFFFFFFFFFFFFFFFFFFFFFFFFFF70
:10208000FFFFFFFFFFFFFFFFFFFFFFFFFFFFFFFF60
:10209000FFFFFFFFFFFFFFFFFFFFFFFFFFFFFFFF50
:1020A000FFFFFFFFFFFFFFFFFFFFFFFFFFFFFFFF40
:1020B000FFFFFFFFFFFFFFFFFFFFFFFFFFFFFFFF30
:1020C000FFFFFFFFFFFFFFFFFFFFFFFFFFFFFFFF20
:1020D000FFFFFFFFFFFFFFFFFFFFFFFFFFFFFFFF10
:1020E000FFFFFFFFFFFFFFFFFFFFFFFFFFFFFFFF00
:1020F000FFFFFFFFFFFFFFFFFFFFFFFFFFFFFFFFF0
:10210000FFFFFFFFFFFFFFFFFFFFFFFFFFFFFFFFDF
:10211000FFFFFFFFFFFFFFFFFFFFFFFFFFFFFFFFCF
:10212000FFFFFFFFFFFFFFFFFFFFFFFFFFFFFFFFBF
:10213000FFFFFFFFFFFFFFFFFFFFFFFFFFFFFFFFAF
:10214000FFFFFFFFFFFFFFFFFFFFFFFFFFFFFFFF9F
:10215000FFFFFFFFFFFFFFFFFFFFFFFFFFFFFFFF8F
:10216000FFFFFFFFFFFFFFFFFFFFFFFFFFFFFFFF7F
:10217000FFFFFFFFFFFFFFFFFFFFFFFFFFFFFFFF6F
:10218000FFFFFFFFFFFFFFFFFFFFFFFFFFFFFFFF5F
:10219000FFFFFFFFFFFFFFFFFFFFFFFFFFFFFFFF4F
:1021A000FFFFFFFFFFFFFFFFFFFFFFFFFFFFFFFF3F
:1021B000FFFFFFFFFFFFFFFFFFFFFFFFFFFFFFFF2F
:1021C000FFFFFFFFFFFFFFFFFFFFFFFFFFFFFFFF1F
:1021D000FFFFFFFFFFFFFFFFFFFFFFFFFFFFFFFF0F
:1021E000FFFFFFFFFFFFFFFFFFFFFFFFFFFFFFFFFF
:1021F000FFFFFFFFFFFFFFFFFFFFFFFFFFFFFFFFEF
:02220000E449AF
:00000001FF
